:020000040000FA
:10000000580A0020292D0000312D0000332D00005A
:1000100000000000000000000000000000000000E0
:10002000000000000000000000000000352D00006E
:100030000000000000000000372D0000392D0000F6
:100040003B2D00003B2D00003B2D00003B2D000010
:100050003B2D00003B2D00003B2D00003B2D000000
:100060003B2D00003B2D0000270400003B2D00002D
:100070003B2D00003B2D00003B2D00003B2D0000E0
:100080003B2D00003B2D00003B2D00003B2D0000D0
:100090003B2D00003B2D00003B2D00003B2D0000C0
:1000A0003B2D0000990200003B2D00003B2D00007D
:1000B0003B2D00003B2D00003B2D00003B2D0000A0
:1000C00000F002F800F0BDF80CA030C80838241881
:1000D0002D18A246671EAB4654465D46AC4201D180
:1000E00000F0AFF87E460F3E0FCCB64601263342F5
:1000F00000D0FB1AA246AB46334318479444000095
:10010000B4440000103A02D378C878C1FAD8520734
:1001100001D330C830C101D504680C6070470000BD
:100120000023002400250026103A01D378C1FBD813
:10013000520700D330C100D50B60704710B56E294F
:1001400002D102F06FFF10BD702902D103F0B1F8A7
:1001500010BD662902D104F0E5F810BD652902D171
:1001600004F0E0F810BD672902D104F0DBF810BDFF
:10017000612902D1C046C04610BD03681B0A01D3E5
:1001800080231943692902D102F016FF10BD6429AA
:1001900002D102F011FF10BD752902D102F00CFF4F
:1001A00010BD6F2902D103F02FF810BD782902D1BC
:1001B00003F06CF810BDE92902D102F0CBFF10BDAD
:1001C000E42902D102F0C6FF10BDF52902D102F0E8
:1001D000C1FF10BDEF2902D103F022F810BDF829AC
:1001E00002D103F061F810BD0368DB0901D380235D
:1001F0001943632902D103F0DAFB10BD732902D140
:1002000003F0DDFB10BDE32902D103F0E7FB10BDD5
:10021000F32902D103F0EAFB10BD002010BD1FB589
:1002200003F044FC04000020002104F065F8401CA9
:1002300060600020002104F049F8E0601FBD10B5A7
:1002400010BD03F00BFC1146FFF7E9FF00F0E3F9E6
:1002500003F0A0FF03B4FFF7F2FF03BC03F0EAFFD3
:1002600070B505460C46164602E00FCC0FC5103E91
:10027000102EFAD2082E02D303CC03C5083E042E5A
:1002800007D301CC01C5361F03E021782970641C17
:100290006D1C761EF9D270BD10B5FE488068022133
:1002A00008404008002850D00220FA49886000BF6A
:1002B000F948C0680446F8480068890308400028E7
:1002C00004D0FF209130844200DA10BDF24800F0E3
:1002D0007CFAF14800F07FFA0020EF49C86000BFC7
:1002E0000846006889030843EB49086000BFEB48F3
:1002F000844202DCEA4884420ADA0020C043E94929
:1003000008600020E84908600120E84908601BE017
:10031000E54800680A2805DAE3480068401CE2491D
:10032000086011E0DB48806820210840400900286F
:1003300005D00120DB490860DD48046004E00020AE
:10034000D8490860DB48046000BF00BFBDE7FEB5C8
:1003500000BFD448066800BFCF48C46800BFD44877
:100360000768D44800680190CE4800688642F0D102
:10037000002E0CDA0021084600F054FC0021022077
:1003800000F050FC0021042000F04CFC4AE000BFCB
:10039000C1488068C007C00F002813D00020C043A8
:1003A000C04908600020C04908600021084600F0EC
:1003B00039FC0021022000F035FC0021042000F06F
:1003C00031FC2FE06420BC490860002E0DD1BC42F6
:1003D00002DBFF25683514E0B42161430846394645
:1003E00002F0E2FC0546B4350BE00198844201DBE3
:1003F000B32506E0B42161430846019902F0D4FC1C
:100400000546A800AD49085800900020009900F06A
:1004100009FC0220009900F005FC0420009900F07E
:1004200001FC00BFFEBD10B5A54800F0D4F9FFF7F0
:100430008EFF10BD70B50024002516E0E800A1492C
:100440000858A04200D26D1CEA009E4BD218516899
:10045000EA00D218526852089B4BD01802F09AFC5E
:10046000401EA100954A5050641CFF206A3084420F
:10047000E4DB70BD1CB5694601A800F01EFE044611
:10048000002C3AD0642C31D00CDC542C2AD004DC63
:10049000202C2DD0462C2FD11DE0562C23D0612CA2
:1004A0002AD121E0762C0AD004DC662C11D0742CE1
:1004B00022D10FE0772C18D0782C1DD117E00198AD
:1004C0008000824A8018006881B281A000F0D0FDCF
:1004D00012E000BF10E0009841100246019800F0C1
:1004E00068FB09E000BF00BF00BF00BF00BF00BF46
:1004F00079A000F0BDFD00BF00BF1CBD10B56E4867
:100500000068002804D06C480068401E6A490860F2
:1005100073480068401C72490860322827D30020C5
:10052000086065480068002802D000206D49C86353
:1005300000206C49403948625C48006800281CD0A3
:1005400000205A49086068480078401CC0B26649DB
:100550000870302803DB08460078392802DD302097
:10056000614908706048007800F008FD05E001204E
:100570005C49C8635B49403948625C4800680028B0
:100580001DD05848006900280BD056484069002803
:1005900007D054488069002803D05248C069002819
:1005A00003D10A205249086034E051480068401ED7
:1005B0004F49086000282DD14C4908602AE049487D
:1005C0000069002806D10120484908600A204849EE
:1005D00008601FE043484069002806D101204349D4
:1005E00008600A204249086014E03E4880690028FB
:1005F00006D101203D4908600A203D49086009E014
:100600003848C069002805D10120384908600A200F
:100610003749086010BD00BF00BF00BF59203549F1
:1006200008601620086088200860084600680028D6
:10063000F4D000BF00F0EBF800BF00202D490860A7
:1006400000BFFFF7F7FE382000F098FC00F027FC11
:1006500000F035FC28484068072109060843264970
:10066000486000F038FB2421002000F086FB482180
:10067000022000F082FB1221042000F07EFB00F03B
:100680007FFA00F071FC1D4800F056FC302000F0AD
:1006900075FC35E000000D4000000140672B0000B4
:1006A0000C1E000004000020100000201400002098
:1006B0000C00002008000020000000205000002056
:1006C00000001140344300004019010000000E40BA
:1006D00025640D0A000000004E410D0A00000000D4
:1006E00018000020C0420050240000201C00002000
:1006F00020000020000100500000044020A107005D
:1007000000F0C1FD192000F051F800F0E3FB4CE0CF
:10071000FFF7B0FE00BF31488068C007C00F002857
:1007200043D02E4800F057F8FFF7E8FE00F0D5FD63
:100730000446002C38DB25D00A2000F03EF828487B
:1007400000F049F8192000F038F8264800F03DF88C
:10075000244800F040F80020C043234908600020EE
:10076000224908600021084600F05CFA00210220BE
:1007700000F058FA0021042000F054FA452000F05F
:10078000FDFB11E0302000F0F9FB164800F01DF8E9
:10079000144800F020F8192000F008F8104800F084
:1007A0001AF80A2000F002F800BFB1E7C206D20E24
:1007B000012191400E4A11607047C206D20E0121FC
:1007C00091400B4A80321160704701680122920704
:1007D0009143016070470121816070470001014031
:1007E0000000114000000140040000201000002023
:1007F00000E100E000BF5920F949086016200860B8
:1008000088200860084600680028F4D0704710B5BA
:10081000042001F0E1FD102001F03EFC0021072042
:1008200001F04AFC012001F0D7FD012001F034FC69
:10083000EC4801F021FD042001F02EFCEA4801F013
:10084000D7FD00221146E84801F05EFDE74801F0BF
:10085000CFFD032252040C21E44801F055FDE44889
:1008600001F0C6FDE34801F0C3FDE34801F0C0FD1F
:10087000002201214902E04801F046FDDF4801F075
:10088000B7FD002201214903DC4801F03DFDDC48B1
:1008900001F0AEFD002201214904D94801F034FDE8
:1008A000D84801F0A5FD002201210907D04801F038
:1008B0002BFD002201214907CE4801F025FDD24839
:1008C00001F036FBD048401C01F032FB0520000748
:1008D000406B000A00020521090748630846406B87
:1008E000332108430521090748630846806B000E41
:1008F000000688630846806BC44908430521090740
:100900008863B748C038806800090001B449C0391D
:1009100088600846806805210843B149C03988606D
:10092000084680680F2109038843AD49C0398860B3
:100930000846806809140843A949C0398860002224
:100940004021B34802F038F9A548C03800680009D2
:100950000001A349C0390860084600680621084321
:100960009F49C039086008460068F02188439C49C7
:10097000C039086008460068602108439849C039BA
:100980000860084600680F21090288439449C0396D
:100990000860084600680321490208439049C039AD
:1009A0000860084600680F21090388438C49C03954
:1009B0000860084600680321490308438849C03994
:1009C0000860084600680F21090488438449C0393B
:1009D0000860084600680321490408438049C0397B
:1009E0000860084600680F21090588437C49C03922
:1009F0000860084600680321490508437849C03962
:100A00000860084600680F21090688437449C03908
:100A10000860084600680321490608437049C03948
:100A2000086005200007C06B0F21090488430521D9
:100A30000907C8630846C06B032149040843052120
:100A40000907C8630846006B0F2109038843052185
:100A5000090708630846006B032149030843052181
:100A6000090708630846006B0F2109028843052126
:100A7000090708630846006B032149020843052162
:100A8000090708630846006BF02188430521090720
:100A900008630846006B60210843052109070863C5
:100AA0000846006B0009000108630846006B062138
:100AB00008430521090708630322102154488030A8
:100AC00002F07AF8032220215148803002F074F8B5
:100AD000032240214E48803002F06EF8032280212C
:100AE0004B48803002F068F80322042148488030E7
:100AF00002F062F803220121C902454802F05CF8C5
:100B00000322FF2101314248803002F055F80322D0
:100B1000012149023E48803002F04EF803220121B3
:100B200089023B48803002F047F803220121C902C4
:100B30003748803002F040F803220121090334488D
:100B4000803002F039F80322012149033048803017
:100B500002F032F80322012189032D48803002F08F
:100B60002BF803220121C9032948803002F024F820
:100B70000322012149022648403002F01DF810BD31
:100B800010B5244800680121084322490860224B1F
:100B90000C2200211F48803800F02EFC01201D4946
:100BA0000861084600680121C90208431949086024
:100BB00010BD10B5062807D2184B84001A51174BE8
:100BC00020338400195109E00C2807D2801F144BF0
:100BD00084001A51124B20338400195110BD0000BB
:100BE0000001005000A24A04113D80571CFE23560C
:100BF0001400C0531500D0530200805E0300C05E95
:100C00000400005F1E0000401400000411111100D8
:100C10004040005080000E403F4000003000044043
:100C20003000144006280FD240084000FA4A8300E2
:100C3000D150431C9B00D1504908F74A2032830011
:100C4000D150431C9B00D150704706280FD240085A
:100C50004000F24A8300D150431C9B00D150490808
:100C6000EE4A20328300D150431C9B00D150704784
:100C700010B500234A0894000246143213514B0069
:100C800003229A4001231B048B401A434368934379
:100C90004360E34B8C0002463032135100238C003A
:100CA00020321351B02212584C00DE4BA3409A431D
:100CB0004C000223A3401A43B0231A50B422125806
:100CC0004C00D84BA3409A434C000123A3401A4345
:100CD000B4231A5010BD10B50021CF483038FFF7AB
:100CE000C7FF0121CC483038FFF7C2FF0221CA48B4
:100CF0003038FFF7BDFF0321C7483038FFF7B8FF92
:100D00000421C5483038FFF7B3FF0521C248303809
:100D1000FFF7AEFF3F21C048303800F07DFE3F2195
:100D2000BD48303800F030FD0021BC483038FFF7B6
:100D30009FFF0121B9483038FFF79AFF0221B748D9
:100D40003038FFF795FF0321B4483038FFF790FFA4
:100D50000421B2483038FFF78BFF0521AF48303807
:100D6000FFF786FF3F21AD48303800F055FE3F21A8
:100D7000AA48303800F008FD10BD70B505460C4695
:100D8000FFF738FDA848844200D904462B0003F041
:100D900070FA060405161726273600BF9E48103045
:100DA000006B01210906884340189B4910310863F4
:100DB000224600219848303800F060FE1FE000BF56
:100DC00095483038406F0121090688434118924800
:100DD000303841672246022100F050FE0FE000BF8C
:100DE0008D483038806F01210906884341188A48B0
:100DF000303881672246042100F040FE00BF00BF6A
:100E000000BF00208949086000BF70BD70B505466D
:100E10000C46FFF7EFFC8448844200D904462B00BF
:100E200003F027FA060405161726273600BF7B486D
:100E30001030006B012109068843401877491031B2
:100E40000863224600217548303800F017FE1FE085
:100E500000BF72483038406F0121090688434118AD
:100E60006E48303841672246022100F007FE0FE04D
:100E700000BF6A483038806F012109068843411855
:100E80006648303881672246042100F0F7FD00BF34
:100E900000BF00BF00206549086000BF70BD10B5ED
:100EA00064220021624801F09BFD61480068000A4D
:100EB000000247305E4908605E48486010BD10B5CA
:100EC00064220121C9065C4801F08AFD5A4800F0FD
:100ED00070FA10BD10B5594A0121C906584801F0F1
:100EE0007FFD00BF56480068012149070843544967
:100EF000086000BF084600F05CFA0021192000F0ED
:100F000021FA0A20012181404E4A116000BF10BD24
:100F100010B54D4A0121C9064C4801F061FD4B480E
:100F20000068000A000247304849086048484860A5
:100F3000084600F03EFA10BD70B5054600240CE0EE
:100F400000BF3D488068C007C00F002805D000BF23
:100F500001203949886000BF641C3E49284601F0E1
:100F600023FFA042ECDC70BD10B53B4800F0E0FF71
:100F7000E1214902394801F083FB10BD01462039C7
:100F8000374A505CC107C90F002903D00021354AF8
:100F9000116202E00121334A11620221014000295D
:100FA00003D000212F4A516202E001212D4A5162F3
:100FB00004210140002903D000212A4A916202E065
:100FC0000121284A916208210140002903D0002113
:100FD000244AD16202E00121224AD162102101405B
:100FE000002903D000211F4A116302E001211D4A9C
:100FF000116320210140002903D00021194A5163C7
:1010000002E00121174A51634021014000292BD001
:101010000021144A91632AE030000440300014405B
:1010200000A24A0403000300FF0F0000000100506B
:1010300000000140CB2B000000010140854501006C
:101040000000114000E100E040420F0000011140AB
:10105000FFFFFF00102700001100000400001540F2
:10106000B4430000C04200500121D54A916370474B
:101070000FB410B5A2B025A80190802102A8019B51
:10108000249A01F06BFE04460020019000BF0DE0A1
:1010900000BFCC4989690122D2051140C90D002940
:1010A000F7D102A9095CC74A1160401CA042EFDBDE
:1010B00022B010BC08BC04B0184710B502460B465D
:1010C000D7E0C0480068C1B20D2901D00A2914D167
:1010D000BD48006804280CDB0020BB4C2060BB48E6
:1010E000407830381060BA4800681860B748007817
:1010F00010BD0020B44C2060BAE0202904D10020AB
:10110000B14C20602020F3E7612901D0412904D1AE
:101110000020AD4C20606120EAE7772901D05729F3
:1011200004D10020A84C20607720E1E7642901D099
:10113000442904D10020A44C20606420D8E77829F9
:1011400001D0582904D100209F4C20607820CFE79F
:10115000462903D0542901D0562905D19B48017056
:101160000120994C206083E09748006801287FDBCC
:101170009848954C2468005D6E2826D1302901DB03
:10118000392903DD0020904C206071E09048006810
:101190000A246043401830388D4C20608B488A4CBC
:1011A0002468015588480068401C874C2060062848
:1011B0005ED3002020608548407830381060844835
:1011C000006818608148007892E782487E4C246865
:1011D000005D6D2830D13F290BD100207A4C206072
:1011E0007A484078303810607848007820242043CE
:1011F0007EE7302901DB392903DD0020724C2060B5
:1012000036E008463038724C206070486E4C2468D6
:1012100001556D480068401C6B4C2060062827D3A0
:1012200000202060694840783038106068480068C5
:101230001860664800785BE76648634C2468005D88
:10124000884212D160480068401C5F4C206006282C
:101250000ED3002020605D484078303810605C4834
:10126000006818605948007842E70020564C20601A
:1012700000BF54488069012189030840002800D13B
:101280001FE7002034E710B500231A460121524819
:1012900001F0C4FC50484068C02188434E49486072
:1012A0000846406807214903884340184A49486076
:1012B0000846406801210903084347494860084639
:1012C0004068032109028843434948600846406852
:1012D000022108434049486010BD4048006881B27F
:1012E0003F4881420ADB3F48006801280FD00120B7
:1012F0003C4A106000203C4A106008E03948006811
:10130000002804D00020374A1060374A1060364861
:1013100000680A2813D234480068401C324A106022
:101320000A280CD1314800682E4A1268904206D033
:101330002C4800682D4A1060104600687047002055
:10134000C043FBE710B5002819DA294A03071B0F31
:10135000083B9B089B00D2588307DC0EFF23A34069
:101360009A438B071B0E8407E40EA3401A43204BBD
:101370000407240F083CA408A4001A5118E01D4AD1
:1013800003231B02D21883089B00D2588307DC0E6C
:10139000FF23A3409A438B071B0E8407E40EA34050
:1013A0001A43144B032424021B198408A4001A5165
:1013B00010BD0168012292071143016070470000CF
:1013C000C0420050000015404000002038000020BE
:1013D000340000200F44000000000D4000000E40CB
:1013E000450700002C0000202800002030000020CD
:1013F0001CED00E000E100E030B580242458494DA8
:101400002C400C43144380252C50842424588425DC
:101410002B5030BD05210907C9680122120711436D
:1014200005221207D1601146C968012212079143B3
:1014300005221207D160704710B500290CD1802316
:101440001B58FF24F134A3430B431343FF240134FF
:101450002343802423501EE010290AD180231B58E7
:10146000FF24F134A3430B430C0123438024235076
:1014700011E09C231B581B0A1B0213439C2423507E
:1014800080231B58FF24F134A3430B43FF24013472
:1014900023438024235010BD80210958FF22F132BC
:1014A0009143802211507047CA07D20F002A05D0FD
:1014B0008022125802231A4380231A5002220A4023
:1014C000002A05D08822125802231A4388231A5072
:1014D00004220A40002A05D08C22125802231A4303
:1014E0008C231A507047CA07D20F002A05D08022D9
:1014F000125802239A4380231A5002220A40002ADB
:1015000005D08822125802239A4388231A500422B5
:101510000A40002A05D08C22125802239A438C23B9
:101520001A507047F3FBFFFFFEB500200290FBA0AE
:1015300000680090FA48046A00132040002801D097
:101540000020FEBD0120C0042040002801D0F54D40
:1015500000E0F54D012040042040002801D028463D
:10156000EFE7032080032040800B69460A5C01926C
:10157000E005C00D861C1F2040022040400A871C49
:10158000019A7A431146AA087243104601F002FC00
:10159000800002900298D4E7FFB583B004460D4660
:1015A0000127E2480090E248844205D1DC484069C6
:1015B000A1020840029005E0D9484069012149078D
:1015C000084002900298002803D1FFF7ADFF0646BD
:1015D0000BE001F037FBD648844203D100F036FD22
:1015E000064602E000F042FD06467D21C900304675
:1015F00001F0D0FB064601271AE0CE4979430846A0
:10160000314601F0C7FB01900599019888420DD23F
:1016100001200003874200D10EE0781CC5494143F8
:1016200001987043814200D806E000E004E07F1C8E
:10163000012000038742E0D900BF781E07466908F1
:101640008A0021461431885060686A000321914065
:1016500088436A000121914008436060606801216D
:101660000904A94088436060AA00214630310098EF
:101670008850019807B0F0BDFFB585B004460D460F
:101680000126AA480290AA48844205D1A44840698C
:10169000A1020840049005E0A148406901214907E2
:1016A000084004900498002803D1FFF73DFF074647
:1016B0000BE001F0C7FA9E48844203D100F0C6FC5B
:1016C000074602E000F0D2FC0746012612E0384649
:1016D000079901F05FFB3146019001F05BFB03903D
:1016E000012109040398884200D902E0039802907E
:1016F00003E0761C90488642E9D300BF029870430D
:101700000146384601F046FB0390701E0646690804
:101710008A00214614318850690003208840012145
:101720000904A94008436168814361600298401E32
:10173000AA002146303102908850029A521C089922
:1017400051430846642101F025FBAA00214650318F
:101750008850B02000596A007849914088436A0057
:10176000022191400843B0210851B42000596A0079
:101770007249914088436A00012191400843B42195
:101780000851039809B0F0BD026A0A43026270472B
:1017900030B5024600200AE0012383400B40002BB5
:1017A00004D000248500134630335C51401C0628C9
:1017B000F2D330BD026A8A430262704730B5042911
:1017C00011D2F8231C58CD000F23AB409C43F823C3
:1017D0001C5080231343CC00A340F82424582343F7
:1017E000F824235012E0FC231B580C1FE5000F24A3
:1017F000AC40A343FC242350802313430C1FE4007C
:10180000A340FC2424582343FC24235030BD10B5AE
:10181000042908D2F8221258CC008023A3409A430E
:10182000F8231A5008E0FC2212580B1FDC0080231A
:10183000A3409A43FC231A5010BD10B501231B048A
:101840008B40FF242134235010BD0246FF2021305D
:10185000805801231B048B401840002801D0012030
:1018600070470020FCE7F0B504460020B6E00125F3
:1018700085400D40002D2FD0812B0CD0822B0AD01B
:10188000882B08D02E4DAB4205D06D1CAB4202D048
:10189000AD1DAB4215D14508AE002546C835AD5942
:1018A000274E7F361E4035434608B6002746C837C8
:1018B000BD51C4252D591E07360F3543C426355159
:1018C0000AE04508AE002546C835AD591D43460817
:1018D000B6002746C837BD51012585401540002D6B
:1018E00048D0C507ED0F002D2CD14508AE00254688
:1018F000C835AD5903263604B5434608B600274619
:10190000C837BD514508AE003D46AD5903263604E3
:1019100035434608B600BD515FE0000001020204F5
:101920000002005000805101001BB700FFFF0000C3
:101930000000044040420F00FF0F000003000300BE
:10194000018000004508AE002546C835AD59032684
:10195000B604B5434608B6002746C837BD5145080A
:10196000AE003D46AD590326B60435434608B600E1
:10197000BD5132E0C507ED0F002D17D14508AE006F
:101980002546C835AD5903263604B5434608B6008A
:101990002746C837BD514508AE003D46AD59012622
:1019A000760435434608B600BD5116E04508AE0042
:1019B0002546C835AD590326B604B5434608B600DA
:1019C0002746C837BD514508AE003D46AD590126F2
:1019D000F60435434608B600BD51401C062800D227
:1019E00045E7F0BD0122520212580A4301235B026F
:1019F0001A501A1D12580A431B1D1A507047012213
:101A0000520212588A4301235B021A501A1D1258BF
:101A10008A431B1D1A507047D82212580A43D823F4
:101A20001A507047D82212588A43D8231A50704748
:101A3000F0B5CC07E40F8F25AD002D584E08F70008
:101A40001E26BE40B5432601D7003E431E43012754
:101A50003E434F08FF00BE4035438F26B600355049
:101A6000F0BD10B58F22920012584B08DC00012304
:101A7000A3409A438F239B001A5010BD30B54B08EA
:101A80009C00034670331B591C0B24034B089D001C
:101A9000034670335C514B089C00034670331B595E
:101AA00001242404144323434C08A5000446703445
:101AB000635130BD10B54A08930002467032D258C7
:101AC00001231B049A434B089C00034670331A51B0
:101AD00010BD10B525231B011B5814468C40234311
:101AE00025242401235010BD10B525231B011B58AC
:101AF00014468C40A34325242401235010BD10B567
:101B000013468B409524A400235010BD10B5024607
:101B1000952080008058FF2301338B401840002817
:101B200001D0012000E00020400095239B009B583D
:101B300001248C402340002B01D0012300E000232E
:101B4000184310BD10B5E0231B5814468C402343A6
:101B5000E024235010BDE0221258DE4B8B409A4304
:101B6000E0231A507047DB4A8A40E8231A50704736
:101B70000246E8208058D74B8B401840002801D0FF
:101B8000012070470020FCE7E422125807238B4015
:101B90001A43E4231A507047E422125807238B405B
:101BA0009A43E4231A5070473F228A40EC231A508C
:101BB00070470246EC2080583F238B401840002895
:101BC00001D0012070470020FCE710B5E0231B582E
:101BD000FF2401348C402343E024235010BDE02235
:101BE0001258FF2301338B409A43E0231A50704769
:101BF000FF2201328A40E8231A5070470246E8204B
:101C00008058FF2301338B401840002801D0012069
:101C100070470020FCE7E022125801238B401A4352
:101C2000E0231A507047E022125801238B409A4358
:101C3000E0231A50704701228A40E8231A50704767
:101C40000246E820805801238B401840002801D02C
:101C5000012070470020FCE770B5F02424584D089F
:101C6000EE007F25B540AC431D018026354315436A
:101C70004E08F600B5402C43F0252C5070BD10B531
:101C8000F02212584B08DC008023A3409A43F02333
:101C90001A5010BD10B5E02212584B08DC0080230A
:101CA000A3401A43E0231A5010BD10B5E022125889
:101CB0004B08DC008023A3409A43E0231A5010BD58
:101CC0004A08D30080229A40E8231A50704710B582
:101CD0000246E82080584B08DC008023A3401840CF
:101CE000002801D0012010BD0020FCE74B08FF2296
:101CF00002329A4003231B02C318DA64704710B5FE
:101D00000246032000021018C06C4C08FF23023367
:101D1000A3401840002801D0012010BD0020FCE79E
:101D200010B5036814468C402343036010BD10B502
:101D3000036814468C40A343036010BDF0B5059CB6
:101D400049084E0003252D02B540012636068E4077
:101D50002E438568B5431E068E40354316024F005C
:101D6000BE40354385608D00064680367451F0BD17
:101D700030B5024600200BE0012383400B40002BCE
:101D800005D0936845080124AC4023439360401C70
:101D90000628F1D330BD30B5024600200BE0012308
:101DA00083400B40002B05D0946845080123AB40CD
:101DB0009C439460401C0628F1D330BD30B50B0520
:101DC00054042343012424041B1984683F256D0413
:101DD000AC432343836030BD8168012212049143E8
:101DE0008160704781680122D2051143816070478C
:101DF00081680122D20591438160704730B5036943
:101E00004C08E5000724AC40A3434C08E500144609
:101E1000AC402343036130BD70B5C0242458CE00CC
:101E20007E25B540AC4315015E0035436D1CCE00E8
:101E3000B5402C43C0252C5070BD10B5C02212589F
:101E4000CC000123A3409A43C0231A5010BD10B503
:101E5000C0221258CC008023A3401A43C0231A503A
:101E600010BD10B5C0221258CC008023A3409A4365
:101E7000C0231A5010BD30B5C0231B58CD0001241B
:101E80002404AC40A343CC0010341546A5402B439A
:101E9000C024235030BD70B5049C15460D43254326
:101EA000FF26193635505D1E361D355070BD024671
:101EB000FF202130805801238B401840002801D09A
:101EC000012070470020FCE701228A40FF232133D4
:101ED0001A5070470000010105210907486070474A
:101EE00005200007806940210840800970470520CF
:101EF0000007406870472B480068C007C00F0121E9
:101F0000484070470520000700687047052000071B
:101F10008068012108430521090788607047052072
:101F2000000780680221084305210907886070477F
:101F3000010E052212078918896801228240114387
:101F4000020E05231B07D2189160010E1A4689184C
:101F50008A68012181408A43010EC9188A6070474E
:101F600005221207926901231A4305231B079A6170
:101F70001A46926908239A43024305231B079A6174
:101F80001A46926906239A430A4305231B079A615E
:101F900070470520000780694008400005210907B7
:101FA0008861704700010050F648806840218843EE
:101FB000F4498860704710B510230B435401234344
:101FC000F04C636223469B6840242343ED4CA3609E
:101FD0002346DB691C24A3430343EA4CE36110BDA1
:101FE000E948006904210843E7490861E5480068B9
:101FF00080210843E349086030BF7047E248006928
:1020000004218843E0490861DE4800688021884354
:10201000DC49086030BF7047DA480068C007C00F6D
:10202000002801D0D94870470020FCE7D548006857
:1020300002210840002801D0880370470020FCE7F7
:1020400010B500F0FFFDD248006810BD10B500F0DB
:10205000F9FDCC48006940210840002803D0CC4855
:102060000068400810BDCA480068FBE710B500F0E2
:10207000E9FDC448006980210840002803D0C44815
:102080000068400810BDC2480068FBE710B500F0CA
:10209000D9FDBF48006810BD0146BE4A05E01046A4
:1020A000521E002801DC00207047B648C068084076
:1020B0008842F4D10120F7E770B504460D46B148D7
:1020C000C068102108400646AE4800680421084355
:1020D000AC4908601020FFF7DFFFAA480069C0087C
:1020E000C000C01DA74908610846806900090001B9
:1020F0002843886108460069C008C0002043086181
:1021000000F0A0FD002E05D19E4800680421884300
:102110009C49086070BD9B48006A0121090408437E
:10212000984908627047F3B589B00C46FFF7F3FF92
:10213000099800280ED1934800680121084391496D
:1021400008600120FFF7A8FF002006908F48089044
:1021500002250EE08B480068042108438949086085
:102160001020FFF799FF0120C00406908A480890CC
:1021700004258A48844204D84010844201D90027AB
:1021800012E08748844205D84010844202D90127D2
:10219000640009E08348844205D84010844202D399
:1021A0000327A40000E057E00020C0430390002074
:1021B0000190029034E02946089800F0EBFD05906C
:1021C0007949059888422AD978490598884226D2C3
:1021D000022007901EE0059E07994E4370488642F4
:1021E00015D34000864212D8A64201D9301B00E028
:1021F000A01B049003990498884208D20498039085
:102200000195079802900398002800D106E00798EE
:10221000401C0790664907988842DCD900BF6D1CB6
:10222000212DC8D9B803069908430199891E49028E
:1022300008430299891E0843524908620420FFF7A7
:102240002BFF781C019A50430146089800F0A2FD2C
:10225000029948430BB0F0BD0998002803D15548B6
:102260004849086202E05448464908620420FFF7E2
:1022700013FF00F019F9EDE770B504464148C06856
:102280001021084005464D48844200D904464C4878
:10229000844200D204463B4800680421084339497F
:1022A00008601020FFF7F8FE364800690721084350
:1022B00034490861084680690009000188610846C0
:1022C000C068C007C00F002805D061000020FFF7DC
:1022D0002AFF04460AE061000120C004FFF723FF43
:1022E00004462848C0681021084005460121022004
:1022F000FFF7E2FE002D05D1224800680421884343
:1023000020490860600870BDF7B586B00022002340
:102310002C4C2546E0CDE46804970396029505947D
:10232000284D103530CD019500948403240E002CE7
:1023300011D00403A40FA4006D462C59114D18357B
:1023400063198403250E8405E40EA5401C68AC4384
:10235000089D2C431C600401640F002C10D08400E5
:10236000A40FA40002AD2C59064D103562190401CA
:10237000650FC401E40EA5401468AC430C4314601F
:1023800009B0F0BD0002005000ED00E0001BB700F6
:102390004400002080F520000080510100C2EB0BBA
:1023A00000E1F50580F0FA02006A18000024F4004C
:1023B000010200002E440000324C080000A24A0432
:1023C00040787D011844000053490969382291433F
:1023D0000143514A116170474F49096801434E4A10
:1023E000116070474C49096881434B4A116070473E
:1023F0000EB54A4B1A6859689B6802930092019186
:10240000810F89006A465158434A89184968C306B2
:10241000DB0E01229A401143820F92006B469A58BC
:102420003D4BD21851600EBD0EB53C4B0C331A68B3
:1024300059689B68029300920191810F89006A4656
:102440005158354A89184968C306DB0E01229A4063
:102450009143820F92006B469A582F4BD2185160CD
:102460000EBD00222E4B1A61042806D11A461269AD
:1024700004231A432A4B1A6106E0274A12693823BB
:102480009A430243244B1A61254A51610022244B8E
:102490009A611A46126903231A43214B1A61704745
:1024A00000201F4908617047FEB5002002901DA062
:1024B000006800901848046A00132040002801D0EA
:1024C0000020FEBD0120C0042040002801D0164D90
:1024D00000E0164D012040042040002801D028468D
:1024E000EFE7032080032040800B69460A5C0192DD
:1024F000E005C00D861C1F2040022040400A871CBA
:10250000019A7A431146AA087243104600F042FC31
:10251000800002900298D4E700020050304400008E
:1025200000E000E00102020400805101001BB7003E
:10253000FEB500200290FBA000680090FA48046AF3
:1025400000132040002801D00020FEBD0120C0045F
:102550002040002801D0F54D00E0F54D0120400459
:102560002040002801D02846EFE7032080032040C8
:10257000800B69460A5C0192E005C00D861C1F2095
:1025800040022040400A871C019A7A431146AA085B
:102590007243104600F0FEFB800002900298D4E7E0
:1025A000012292020A40002A01D06822826101229F
:1025B000D2020A40002A03D0426901231A43426131
:1025C000012252030A40002A01D0DA4A8261012224
:1025D00092030A40002A01D0426C42640122D203D5
:1025E0000A40002A03D08022C261826B8263704756
:1025F000002141607047416803221203914341600A
:10260000704770B504460D466068A8436060CA48CC
:10261000844203D10C2000F0A2F909E0C7488442AB
:1026200003D10D2000F09BF902E00C2000F097F997
:1026300070BD0169012252021143016141695210CA
:102640001143416141680322120311434160704705
:1026500070B504460D46606828436060B648844201
:1026600003D10C2000F074F909E0B448844203D18E
:102670000D2000F06DF902E00C2000F069F970BD4A
:10268000F0B587B004460D46AD4801460EC9C06896
:1026900003AE0EC6069000200290A34840690321B5
:1026A00009060840060EA04880690F21090208406B
:1026B000070A002020630320E060A068A1490840C9
:1026C000A060012E04D1FFF733FFB10003AA5050E0
:1026D000002D26D0B10003AA5058791C00F05AFBF7
:1026E000690840182946019000F054FB801E0290B2
:1026F0009549029888420FD9B10003AA5058791C15
:1027000000F048FBE90040182946019000F042FB28
:102710000009801E606204E0032109070298084353
:10272000606207B0F0BD70B503460C46002111E0B1
:10273000002506E06D1C01208007854201D30020A2
:1027400070BD98690126B60330400028F2D11868A0
:102750006054491C9142EBD30846F1E7FFB587B0BE
:1027600004460D4617467648103001460EC9C0682B
:1027700002AE0EC60590002001906B48406903210F
:1027800009060840060E684880690F2109020840C2
:10279000000A0690012E04D1FFF7CAFEB10002AA7A
:1027A0005050002D28D0B10002AA50580699491C5B
:1027B00000F0F0FA690840182946009000F0EAFAA3
:1027C000801E019060490198884210D9B10002AA88
:1027D00050580699491C00F0DDFAE90040182946D6
:1027E000009000F0D7FA0009801E606204E0032127
:1027F000090701980843606238460A99084310990E
:102800000843E0600BB0F0BD026A120A12020A43EC
:10281000026242680123DB021A4342607047F7B547
:1028200086B004460E464648203001460EC9C068B0
:1028300001AD0EC50490022020633B48406903218E
:1028400009060840070E384880690F210902084030
:10285000000A0590012F04D1FFF76AFEB90001AA12
:102860005050002E12D0B90001AA50580599491CA9
:1028700000F090FAF10040183146009000F08AFA1A
:102880000009851E3048854200D2656208980028FC
:1028900008D1A06A40210843A062A06A02218843AF
:1028A000A06207E0A06A20218843A062A06A0221FA
:1028B0000843A06209B0F0BD10B503230363C36AE7
:1028C000224C2340C362C36A14060C432343C362F1
:1028D00010BD10B501230363C36ACF24A343C362B1
:1028E000C36A0C4614432343C36210BD70B503464C
:1028F0000C46002111E0002506E06D1C0120800738
:10290000854201D3002070BD98690126360730400A
:102910000028F2D0605C1860491C9142EBD1084657
:10292000F1E70000010202040002005000805101A2
:10293000001BB70001000001000005400000154029
:10294000484400000FFFF0FFFFFF0000FFF8FF000A
:10295000C206D20E01219140054A11607047C2069D
:10296000D20E01219140024A80321160704700006E
:1029700000E100E030B589B005462022824901A877
:10298000FDF76EFC8148854206D1814840690721E8
:1029900009020840040A19E07E48854206D17C48B5
:1029A0004069072109030840040B0FE07A4885427B
:1029B00006D177484069072109040840040C05E066
:1029C00073484069072109050840040D022C03D112
:1029D0007248006809B030BDA00001A90858F9E7A5
:1029E000F7B582B0064617463046FFF7C3FF0190A1
:1029F0000024002501984008B84201D202240CE0CE
:102A00003946019800F0C6F90446250E002D04D081
:102A1000691C204600F0BEF9044603982843306044
:102A20007460681C60430146019800F0B3F905B07A
:102A3000F0BD0021016041617047FEB505460C46BE
:102A40002846FFF797FF0746002002903946534873
:102A5000006800F09FF9401C019000202860686128
:102A60004F48874209D87D20C000844200D20446E6
:102A70004B48844208D9044606E0642C00D2642402
:102A80004748844200D90446454887420FD8002071
:102A900002903946434800F07DF900907D21C9003D
:102AA00061430846009900F075F9064610E03C497C
:102AB000384600F06FF906466643300E02900298E1
:102AC000002805D00299491C304600F063F90646FB
:102AD0006E600121890702980843286003E000BF67
:102AE0000198401E019001980028F8D100BF286885
:102AF0000121490608400028F9D1FEBD10B54369FF
:102B0000294C23400B43134308242343436110BD46
:102B1000416908229143416170474269520852005D
:102B20000A434261026801231B061A430260704790
:102B300001680122120691430160704730B50C46CE
:102B4000124DA84201D1134D00E0184D2946184DF1
:102B50004D60002B01D0202500E000254D61154D72
:102B6000056030BD01680122D204914301607047C5
:102B7000C269520852000A43C2617047C2691623F3
:102B80009A430A43C2617047784400000000014044
:102B900000020050000101400000114044000020EC
:102BA00040420F0000CA9A3BEF8FFFFF0001114027
:102BB000FFFFFF000000084070B5034600200FE053
:102BC000012484400C40002C09D01C6846000325D9
:102BD000B540AC4346001546B5402C431C60401C34
:102BE0001028EDD370BD10B58469130E8B401C43C3
:102BF0008461C3691402240A8C402343C36110BD5D
:102C0000826901238B409A438261C369024A8A40E8
:102C10009343C361704700000100010070B58C0050
:102C200004593425AC4315461D43012635432C4336
:102C30008D00445170BD8A008258520852008B00AA
:102C4000C250704770B52F48006945076D0F00F0FE
:102C500020F82D490860022D03D0A8002B490C58FC
:102C600001E029480468274880690007000F461CD6
:102C70003146204600F08EF8254908602549244851
:102C800000684A10801800F085F82349086070BD7C
:102C90007047FEB50020029020A0006800901948FF
:102CA000046A00132040002801D00020FEBD01204E
:102CB000C0042040002801D0194D00E0194D01202A
:102CC00040042040002801D02846EFE7032080037D
:102CD0002040800B69460A5C0192E005C00D861C0D
:102CE0001F2040022040400A871C019A7A43114667
:102CF000AA087243104600F04DF880000290029836
:102D0000D4E70000000200504C000020984400006E
:102D10004400002040420F0048000020010202044D
:102D200000805101001BB700074880470748004753
:102D3000FEE7FEE7FEE7FEE7FEE7FEE7044805499B
:102D4000034A054B70470000912C0000C1000000B1
:102D500058060020580A0020580600207CB51D4661
:102D600016460C00009001D00019401E084B7B4411
:102D70002A4669460190304600F06DF9002C054660
:102D800003D06946002000F079F928467CBD000098
:102D900015030000002203098B422CD3030A8B4247
:102DA00011D300239C464EE003460B433CD4002243
:102DB00043088B4231D303098B421CD3030A8B4255
:102DC00001D394463FE0C3098B4201D3CB01C01A23
:102DD000524183098B4201D38B01C01A52414309EE
:102DE0008B4201D34B01C01A524103098B4201D3DC
:102DF0000B01C01A5241C3088B4201D3CB00C01A49
:102E0000524183088B4201D38B00C01A52414308C0
:102E10008B4201D34B00C01A5241411A00D20146E5
:102E20005241104670475DE0CA0F00D0494203107E
:102E300000D34042534000229C4603098B422DD3CD
:102E4000030A8B4212D3FC22890112BA030A8B4275
:102E50000CD3890192118B4208D3890192118B42C4
:102E600004D389013AD0921100E08909C3098B4249
:102E700001D3CB01C01A524183098B4201D38B018C
:102E8000C01A524143098B4201D34B01C01A52412F
:102E900003098B4201D30B01C01A5241C3088B4274
:102EA00001D3CB00C01A524183088B4201D38B005F
:102EB000C01A5241D9D243088B4201D34B00C01AE9
:102EC0005241411A00D20146634652415B101046FE
:102ED00001D34042002B00D54942704763465B1046
:102EE00000D3404201B50020C046C04602BD704735
:102EF0007047704770B5044685690068C10601D502
:102F0000302600E02026C00707D070BD626830463A
:102F1000A1689047206A401C20626D1EF6D570BDE6
:102F200070B5044685690078C00707D170BD626836
:102F3000A16820209047206A401C20626D1EF6D5B3
:102F400070BD09684A0501D540B27047C905FCD576
:102F500000B2704709684A0501D5C0B27047C9057B
:102F6000FCD580B2704770B50C460546012A05D0E5
:102F70002878800600D5EA69002302E0012305E0F5
:102F80005B1C934202D2E05C0028F9D1A869E618E4
:102F9000C01AA861286AC01828622846FFF7AAFF4D
:102FA00004E06A682078A968641C9047B442F8D3AA
:102FB0002846FFF7B5FF70BDF7B5002575291068E5
:102FC000009914A611D0FFF7BCFF002802DA404296
:102FD00011A608E0009909688A0701D50FA602E04A
:102FE000490704D50EA6012501E0FFF7B3FF009FB6
:102FF0000024243704E000F01DFD30313955641CF5
:103000000028F8D12B4632462146009800F05FFA9E
:10301000FEBD0000000000002D0000002B0000009D
:103020002000000011680268006A530501D508708D
:1030300009E0D30501D5088005E0130602D5C217C3
:1030400005C100E0086001207047000001694A1CCA
:1030500002610878704700B58FB002910021059198
:10306000054901937944039111460490684600F0A4
:103070002DF90FB000BD0000E5FFFFFF0A681070DA
:10308000521C0A6070470CC908399A4202D2531C7C
:103090000B60107070470000F7B50446154686B007
:1030A0002B487844002703C83E460090019111E068
:1030B00007986A467100415A02A800F09BFC411C27
:1030C00007D02178890603D5E269391891420ED8D4
:1030D0003F18761C2078800602D5E069B84206DDEC
:1030E000AE42E5DB07987100405A0028E0D1A069A4
:1030F000C01BA0612046FFF7FDFE154878445A38F2
:1031000003C800900020019116E041006A4607982C
:10311000415A02A800F06EFC0590401C0AD0002520
:1031200005E0626802A8A168405D90476D1C0598A3
:103130008542F6D30498401CB0420490E5DB206A37
:10314000C01920622046FFF7EBFE09B0F0BD000079
:1031500012140000F7B5D21D0025D20815A6D20022
:10316000F52905CA11D0002A05DA00214042914113
:1031700011A60A4608E0009909688B0701D50FA639
:1031800002E0490701D50EA601251146009F002443
:10319000243704E000F05EF930323A55641C0246F0
:1031A0000A43F7D12B4632462146009800F08FF9AA
:1031B000FEBD0000000000002D0000002B000000FC
:1031C0002000000070B504460021243408E05507B3
:1031D000D2086D0F303565545D072A43DB08491C62
:1031E00015461D43F3D10468002310A2250708D516
:1031F000A40601D4002904D0C46901230CA2641ED2
:10320000C46100F064F970BD10B504462146106831
:10321000FFF7A0FE002302462046FFF7D3FF10BDB4
:10322000D21DD108C9000CC9CCE700000000000085
:1032300030000000F8B50F460188090502D5224C80
:103240007C4402E0204C7C440E34054600212435A9
:1032500008E016071209360FA65D6E541E073243AA
:103260001B09491C16461E43F3D12246047800234D
:10327000240705D5702F06D0002901D00223113272
:1032800000F025F9F8BD01231032F9E770B50446C6
:103290000D4621461068FFF75DFE002302462946D1
:1032A0002046FFF7C7FF70BDD21DD308DB000CCB53
:1032B000C0E730B403682024126823430360082366
:1032C000C36130BC0023B5E77C120000F3B50446AF
:1032D000002081B020622046E1688847002872D033
:1032E000252802D06268A168ABE0594F00267F44D0
:1032F0002046E16888472028054608DB312D06D2A4
:10330000781920380078002801D00643F0E7B0078C
:1033100001D5042086430020E0610746A0612A2DE4
:103320000AD0284600F0CAFF002827D0B8000019AC
:10333000303D0090856119E00298BA00121902C868
:10334000916102902046E1688847012F054617D118
:10335000E06900281FDA202086431CE000980A213B
:103360008069484300994019303888612046E168F7
:103370008847054600F0A2FF0028EFD1012F0AD0B0
:103380002E2D08D12046E1688847054620200643B7
:103390007F1C022FC3DBA069002803DA4042A06132
:1033A00001200643F00701D0102086436C2D0BD07E
:1033B000682D09D04C2D3CD06A2D38D0742D38D0D2
:1033C0007A2D36D016E040E0E1682F462046884747
:1033D000B842054609D16C2F29D001208002E1684E
:1033E000064320468847054604E06C2F1DD0FF2089
:1033F00001300643002D28D028464138192803D82B
:103400000120C00206432035204626602946029A44
:103410001646FCF793FE002810D001280BD0F61DAD
:10342000F008C0000830029055E74020E1E7802016
:10343000D5E70020D3E7361D02964CE762682846A0
:10344000A1689047206A401C44E7206AFEBD000046
:10345000F61100000B4670B5024689078008084344
:1034600019469D08141AA9412509080705430809AA
:103470002C194841250A01060D43010A2C19414126
:10348000200C0D0428430D0C00194D41002140195A
:103490004D41C00869070843E908840F8D002543A2
:1034A000840024184D4124196D41121BAB4107E0E3
:1034B0000925ED432C11521963410024401C614140
:1034C0001C460A250026551BB441F1D270BDFFB53C
:1034D00004460D4681B0243000902168880604D54A
:1034E0001022E0699143216000E00120A84201DD43
:1034F000471B00E000270498A1697A191018081AE0
:10350000A0612078C00602D42046FFF7F3FC002615
:1035100008E003986268A168805D9047206A401CBB
:10352000761C206204988642F3DB2078C0060AD518
:103530002046FFF7DFFC06E06268A1683020904774
:10354000206A401C206238467F1E0028F4DC07E019
:1035500000986268A168405D9047206A401C206224
:1035600028466D1E0028F3DC2046FFF7D9FC2078A2
:10357000000602D5022005B0F0BD0120FBE70000E7
:103580007047FFB50C461E468FB003CA08900991DC
:103590004F007D0D00D16D1E002108460020C04661
:1035A0000321099A89050840002A03DA820080185D
:1035B00040080840800D01280A9002DD0020C04329
:1035C0000A90089807430DD0F048F149281848435D
:1035D0000714189800281DD07542291E1DDD0A9871
:1035E00042421BE01898012802D00020302104E05C
:1035F0000020F24305E02154401CB042FBDB304682
:103600000022189B002121540F998B600A604860AA
:1036100013B0F0BDBD1B6D1CDFE70A9A002900DA6C
:1036200069420BA800F08AFA0BAB07CB03AB07C3C8
:103630000899099800F0EEFA6B4607C30146D54891
:103640000918002D00910BDDD24903980A9A4942CE
:103650004018002303A90390684600F04BFD08E0E2
:1036600003990A9A0023081803A90390684600F0FA
:10367000EBFC6B4607C30004000C03D00020C043E2
:10368000410800E01046189A002A03D00022009258
:1036900015461EE0751E05D4FFF7DCFE303262557C
:1036A0006D1EF9D501220843079602D000227F1C27
:1036B00004E02078302801D100227F1E002A0697DE
:1036C00087D01EE0112D07DAFFF7C4FE30326255B5
:1036D0006D1C02460A43F5D1084303D00098002828
:1036E00019D00EE00021681E05E0235C625C635483
:1036F0002254401E491C8142F7DBA81B401E07953F
:103700000690079A18990020A0540F98079B069AD4
:1037100081600CC07CE711260020189059E7D21D6B
:10372000F0B50D460446D10893B0C90003C90C900A
:103730000D9100F0ADFD02460D98C00F01D02D2077
:1037400007E02068810701D52B2002E04007C00F69
:103750004001032A0F9001D0072A05DB03462946C2
:10376000204600F0A7F90EE12078800601D5E76930
:1037700000E006272846652D04D0662814D0672D62
:1037800069D12DE00020112F009001DB112300E012
:103790007B1C0CAA03A910A8FFF7F3FE11990026C1
:1037A00010987D1C0E9142E001203B460CAAC007F8
:1037B0000B900120009003A910A8FFF7E2FE119DD5
:1037C00012981099002600280E9501D1781C0D182A
:1037D000781B02D446427D1C761EE81B00903AE01E
:1037E000012F00DA01270020112F009001DD1123A5
:1037F00000E03B460CAA03A910A8FFF7C2FE1199EE
:103800003D46109800260E91217809070BD40E9999
:10381000A94200DA0D4603A9012D04DD4A19203A18
:10382000D27F302A06D0B84201DA011D04DA012124
:1038300000910FE06D1EEFE7002802DC86192D1ABB
:1038400003E0411CA94200DD0D46801B401C009096
:103850000120C0070B902078000705D40098A842EB
:1038600002DB0020C043009069460020C8720B981C
:10387000012102AF0337C907884225D002201090EA
:103880002B2011900B9800280BDA40420B902D2032
:10389000119006E00B9800F0CDF830317F1E0B90B0
:1038A00039701099481E00291090F3DC0B980028FD
:1038B000F0D111987F1E38702088000501D5452071
:1038C00000E065207F1E387001A8C01BC01D0B9052
:1038D0000F98002800D0012041190098C01709183E
:1038E0000B980818A169081A401EA0612078C0062C
:1038F00002D42046FFF7FEFA0F98002805D0626830
:10390000A1689047206A401C20622078C00625D517
:103910002046FFF7EFFA21E0002E07DB0E98B042B9
:1039200004DD03A86268805DA16802E06268A168A6
:1039300030209047206A761C401C20620098401E70
:10394000002800900AD100F0B1F8C06862680168F0
:10395000405CA1689047206A401C206228466D1E8A
:103960000028D9DC07E062683878A1687F1C90479E
:10397000206A401C20620B99481E00290B90F2DC43
:103980002046FFF7CDFA032042E6000001FCFFFFCE
:10399000104D0000E1DFFFFF10B54369002B02D09E
:1039A000C046C04601E0FFF7DEFA012010BD1278E4
:1039B000014624310A7000224A700122ECE71168A6
:1039C0000022D243E8E710B54369002B02D0C0467D
:1039D000C04601E0FFF760FB012010BD12880146E0
:1039E000243182840022C2840122ECE71168002283
:1039F000D243E8E770B516460C46054600F04EF88F
:103A00000368FF200230C05C012807D0FF2C0ED8CD
:103A1000185D00280BD001202C7070BDFF3332469A
:103A2000214608331868C3182846984770BD0020FF
:103A3000C04370BD01468008081A02091018020A26
:103A40001018020C1018C008820012185200891AAF
:103A500001E0401C0A390A29FBD27047754600F084
:103A6000A1FBAE46050069465346C008C000854626
:103A700018B020B5FFF762F960BC00274908B646C8
:103A80000026C0C5C0C5C0C5C0C5C0C5C0C5C0C56D
:103A9000C0C5403D49008D467047000010B500F09C
:103AA00005F8001D10BD00BF510800000048704718
:103AB00014060020F8B51F46044601230068DB0207
:103AC000032601461840072A05DB002801D017A568
:103AD00006E017A504E0002801D016A500E016A511
:103AE000102081432160A069C01E002FA06101D079
:103AF000401EA0612046FFF7FDF9002F09D038468F
:103B00006268A1689047206A401C2062C01C206245
:103B100006E0206AFAE762682878A1686D1C904781
:103B2000761EF8D22046FFF7FBF9F8BD4E414E0055
:103B30006E616E00494E4600696E6600F7B5164626
:103B40008AB0334878446C4603467C33C06F5A6869
:103B50009B680DC42E487844763003AC0DC80DC464
:103B60003720C001081837211B30FFF71DF9054623
:103B70000C46803D1B3C02D56442012000E0002041
:103B80000027099010E0E0070CD00C202049784372
:103B9000794432464C3941186846012300F054FA02
:103BA0006B4607C364107F1C002CECD1184F7F4478
:103BB0002E3F16E0E80712D02001C0190EC806916A
:103BC000089307920068F04201D198190890324694
:103BD000012306A903A800F037FA03AB07C36D1051
:103BE000641C002DE6D10998002806D032466946AB
:103BF000012303A800F07EFA05E00123324669465E
:103C000003A800F021FA0A9B07C30DB0F0BD000025
:103C1000B4090000034640000A4610B5400D0BD021
:103C20000121C9070F24A40200191C0364082143C1
:103C3000540D2143D20207E000210120F2E7D40F06
:103C4000490021435200401E0029F8DADB0FDB0750
:103C5000184310BDFFB50D46144685B0486851683D
:103C600000F0EFFA00910190A868A16800F0E9FA6D
:103C700002910390A868616800F0E3FA029A1218B2
:103C80008242029201D2012000E00020019A0B182A
:103C9000D2180028019202D08A4202D903E08A4257
:103CA00001D2012000E00020009908180090686807
:103CB000A16800F0C6FA029A12188242029201D25A
:103CC000012000E00020019A0B18D2180028019270
:103CD00002D08A4202D903E08A4201D2012000E0E8
:103CE00000200099081800902868216840004900C9
:103CF000400849084018FA49471814E00199400063
:103D0000C90F08430090019802994000C90F084369
:103D10000190029803994000C90F0843029003984C
:103D200040007F1E039000980028E7DA08980028DA
:103D300001D0EC4E00E00026B74201DA012000E09D
:103D40000020002804902AD0F71BF806C00E15D0DA
:103D5000029B2021091A039A8B401A430392029A6C
:103D6000019BC2408B401A430292019A009BC240C1
:103D70008B4000991A430192C14000917B110DD0F4
:103D80006F460320C11A03D500218200B95003E019
:103D90008A008100BA587A50401EF3D537460398FE
:103DA0000299002800D001200143089802910028C0
:103DB00008460CD0002800D001200199019A49053D
:103DC00008430121D20AC902D202019200E0012176
:103DD0000E9B0122D207012B02D0002B03D013E04F
:103DE000002807D120E0904204D890420CD1019BDA
:103DF0000B4209D0019B5918019105D10099491C2A
:103E0000009101D17F1C009200280DD0102108469E
:103E10000020C0460498002806D00F98002803D040
:103E2000082108460020C04628682168019B009AA6
:103E30004840C10F0598C90739430EC009B0F0BD0D
:103E4000FFB587B0099A0898089953689268406846
:103E5000896896460022039317469446089A12688A
:103E60005300099A5B081268520052089A1A9E4B36
:103E7000D4180A9A002A01D0352200E04022069286
:103E80000022012315460492DB07059324E0002D50
:103E900005D175460346039E4D1BB34109D37546B4
:103EA0006646039B491B049D9841059B7519AC46CA
:103EB0005F4163463B4308D0059B049EDD077608BF
:103EC0002E435B080496059301E0521E641EC50F45
:103ED000ED0749184041521C069B9A42D7DB002D42
:103EE00004D17546039A6B1A824101D203200CE07B
:103EF000039A0B466B404240134303D0014303D067
:103F0000012002E0022000E0002061460191002132
:103F1000009702910A99002905D0614640020143A9
:103F2000704B019102E08007002302909C4201DA6D
:103F3000012000E0002007003AD01A1BD006C00E76
:103F400015D0029D2021019C091AC5408C402543B3
:103F5000029C8C4000D001242543019C0295009DC9
:103F6000C4408D4000992C430194C14000915411EC
:103F70001DD06D460221002202290CD10320001B16
:103F800007E0002804DB8600AE59002E00D0012295
:103F9000401C0328F5DB081B02D588002A5004E0EA
:103FA0008000285810438A00A850491EE3D51C46BB
:103FB0000A98002802980CD0002800D0012001990E
:103FC000019A490508430121D20AC902D20201928D
:103FD00000E00121109B0122D207012B02D0002B0F
:103FE00003D013E0002807D11FE0904204D890428C
:103FF0000CD1019B0B4209D0019B5918019105D1AD
:104000000099491C009101D1641C009200280CD039
:10401000102108460020C046002F06D01198002825
:1040200003D0082108460020C04608980999019A43
:10403000009B006809684840C10F0798C9072143E1
:1040400082600AC00BB0F0BD00B585B0019300924C
:104050000A460146002302A8FFF7FCFD02A807C894
:1040600005B000BDFFB50A461F4685B0079901930C
:1040700001230091014602A8FFF7ECFD0299039885
:10408000049ECA0F4900D20700920F2249089202EB
:104090008C1A0021002800DB0C46450013486D08EF
:1040A000844214D3079A002A04DA441E0026104DD5
:1040B000F64302E004460D460E4610210846002055
:1040C000C046002F03D0042108460020C04620052A
:1040D000E90A0843009908436905F20A1143ADE66D
:1040E00002C0FFFF013C0000FF3F0000FF0700008F
:1040F000FFFFFF7F00B585B0019300920A4601469D
:10410000002302A8FFF79CFE02A807C8A8E7FFB596
:104110000A461F4685B00799019301230091014685
:1041200002A8FFF78DFE02990398049ECA0F49006A
:10413000D20700920F22490892028C1A002100280F
:1041400000DB0C46450011486D08844214D3079AE1
:10415000002A04DA441E00260D4DF64302E0044610
:104160000D460E46102108460020C046002F03D001
:10417000042108460020C0462005E90A08430099AA
:1041800008436905F20A114358E60000FF070000E2
:10419000FFFFFF7F10B50446C046C0462046FCF72F
:1041A00059F810BD00487047F4050020024670B56C
:1041B0000A4392072AD11E4DEE0104C808C9541BB8
:1041C0009443344017D0D0B2D9B2401A21060143EB
:1041D00010D190B299B2401A210401430AD11002C1
:1041E0001902000A090A401A2102014302D1100EE5
:1041F000190E401A70BD9A42DFD010BA19BA88421F
:1042000001D9012070BD0020C04370BD02780B7839
:10421000401C491C002A09D09A4207D102780B7829
:10422000401C491C002A01D09A42EFD0D01A70BD20
:104230000101010101491820ABBEFEE72600020082
:104240007047F8B5040C8BB2264682B25E43104626
:1042500058430D0C370C360400218019164679415D
:104260006E43370C36048019264679416E4389190E
:10427000F8BD30B47446641E2578641CAB4204D388
:10428000635D5B00E31830BC18471D46F8E700008B
:104290004900CA020243100000D004204A0D01D098
:1042A00001221043044A490D914201D102210843E1
:1042B000012800D105207047FF07000030380A2888
:1042C00001D20120704700207047000010B500297E
:1042D0000AD00878002807D005487844FFF766FF21
:1042E000002801D0002010BD0248784410BD000015
:1042F000D6020000CE02000010B500290AD00878CE
:10430000002807D005487844FFF750FF002801D067
:10431000002010BD0248784410BD0000C602000015
:10432000BE02000003B402487844844603BC6047E0
:10433000F3F3FFFF1E0000003C000000320000000D
:104340005000000046000000640000005A00000019
:10435000960000006E000000960000008200000041
:10436000640000009600000050000000B40000004F
:104370003C000000D20000003C000000E60000000D
:1043800050000000FA000000640000000E01000070
:104390009600000022010000960000003601000097
:1043A000640000004A0100005000000068010000A5
:1043B0003C000000003022416D527C20390F2170FA
:1043C000084080523F065B4F666D7D077F6F48480F
:1043D00039480F535F777C395E79713D76061E76DA
:1043E0003815373F7367316D786E1C2A766E5B39EE
:1043F000640F230820777C585E79716F74041E76F1
:104400001815545C7667506D783E1C2A76675B46BB
:104410006E3D6D6E6E0000000000000004000000A4
:104420000C0000002400000000000000200000003C
:1044300000000000040000002C000000000000004C
:10444000040000002C000000001BB700000000006A
:104450000080000000805101001BB7000000000038
:104460000080000000805101001BB7000000000028
:104470000080000000805101001BB7000080000098
:1044800000000000000000000000000010270000F5
:104490000000000000805101001BB70000800000F8
:1044A00000E0480410270000006CDC02000000005F
:1044B000000000000080510100000000000000002A
:1044C000303132333435363738394142434445464A
:1044D0004030580030313233343536373839616244
:1044E0006364656640307800040000080000000046
:1044F0000000000200010000100000000240000067
:10450000000000A00000000005400000000000C8FE
:10451000000000000C4000000000409C0000000073
:10452000194000000020BCBE000000003440000024
:10453000BFC91B8E00000004B5400000504BCFD017
:104540006607E2CF010000006C4100003E8251AAE4
:10455000DFEEA73401000000D9420000DCB5A0E284
:104560003A301F97FFFFFFFFB4450000FD25A0C8AC
:10457000E9A3C14FFFFFFFFFFF3F000000000080E5
:1045800000000000FF3F000000000080000000006D
:10459000DC46000000000020500000000401000084
:1045A0002C47000050000020080A000020010000F5
:1045B0001C00000043000000F8FFFFFF0C0000009B
:1045C0000E0000000F0000002E000000100100008F
:1045D00043000000F8FFFFFF0040404040404040E3
:1045E00040404141414141404040404040404040C6
:1045F000404040404040404040050202020202026A
:1046000002020202020202020220202020202020B8
:1046100020202002020202020202909090909090CC
:10462000101010101010101010101010101010108A
:1046300010101010020202020202888888888888FE
:1046400008080808080808080808080808080808EA
:1046500008080808020202024000000000000000F2
:10466000000000000000000000000000000000004A
:10467000000000000000000000000000000000003A
:10468000000000000000000000000000000000002A
:10469000000000000000000000000000000000001A
:1046A000000000000000000000000000000000000A
:1046B00000000000000000000000000000000000FA
:1046C00000000000000000000000000000000000EA
:1046D00000000000000000000000000000000000DA
:1046E000FFFFFFFF000000000000000000000000CE
:1046F00000000000000000000000000000000000BA
:104700000000000000000000FFFFFFFF00000000AD
:104710000000000000000000000000000000000099
:0C47200000E048044700000000E04804EE
:0400000500002D29A1
:00000001FF
